:040500002FEF24F0C5
:08050800046ED8CF05F0E0CF2E
:1005100006F00001E9CF0CF0EACF07F0E1CF08F0D8
:10052000E2CF09F0D9CF0AF0DACF0BF0F3CF12F017
:10053000F4CF13F0FACF14F0F5CF15F0F6CF16F094
:10054000F7CF17F0F8CF18F0FBCF19F000C00EF07E
:1005500001C00FF002C010F003C011F09DA6B4EF6F
:1005600002F09EB62DEF03F00EC000F00FC001F0B8
:1005700010C002F011C003F00CC0E9FF07C0EAFF91
:10058000078E08C0E1FF09C0E2FF0AC0D9FF0BC017
:10059000DAFF12C0F3FF13C0F4FF14C0FAFF15C056
:1005A000F5FF16C0F6FF17C0F7FF18C0F8FF19C017
:1005B000FBFF045006C0E0FF05C0D8FF10000A0191
:1005C000EE6B020179517B5D03E17A517C5D33E092
:1005D0007D0E7B25E96E060E7C21EA6EEFCFEEFAEA
:1005E0000A01010E02017B250A01EF6F000E0201D4
:1005F0007C210A01F06F030804E202017C6B7B6B33
:1006000004D002017B2BD8B47C2B0A01EE3D03D031
:100610007E5301E07E07020179517B5D07E17A514B
:100620007C5D04E10A017F9397988E880A01EECAE7
:1006300001F004D00201FF0E016E0A01000162EF19
:1006400003F0C950EFCAC9FFC6889E96C7B0FED74F
:10065000016AC6B8012A67EF03F0C7B432D07D0E35
:1006600002017525E96E020E7621EA6EC69C9EA6F1
:10067000FED7C950C688EF6EC7AA21D07D0E75255A
:10068000E96E020E7621EA6EEF3C03D00A017D2B63
:100690000201010E75250A01EE6F000E020176219E
:1006A0000A01EF6F030805E30201752BD8B4762B1E
:1006B00003D00201766B756B0A017F81020108D0BD
:1006C00000017DD701C0EEFA01C0EFFABAD70201EE
:1006D0009E960001B4EF02F00A018F6B8E6B7D6B6A
:1006E000806B02017A6B796B7C6B7B6B766B756BC5
:1006F000786B776B0A018F6B8E6B8F51030812E357
:100700007D0E8E25E96E020E8F21EA6EEF6A7D0E58
:100710008E25E96E060E8F21EA6EEF6A8E2BD8B415
:100720008F2BEBD7000127EF28F00A01E06BDF6B7E
:10073000DE6BDD6BE46BE36BE26BE16BE66BE56B51
:10074000E86BE76BEA6B180EE96FD9CAE0FADACA10
:10075000DFFADBCADEFADCCADDFA95988C9800D0A5
:1007600000D0E86B080EE76FE66BE56BE65320E11F
:10077000E55107081DE3E751D8B4E807E707959A64
:100780008C9AD9CA00F0E751016E04E0D89000328B
:10079000012EFCD700B002D08C9C01D08C8C959C93
:1007A00000D0959A8C8A00D0E52BD8B4E62BDED702
:1007B000E86B080EE76FE95F000EEA5BE66BE56B3E
:1007C000E65340E1E55107083DE3E751D8B4E807B7
:1007D000E707959A8C9ADACA00F0E751016E04E0B7
:1007E000D8900032012EFCD700B002D08C9C01D0F2
:1007F0008C8C959C00D0959A8C8A00D0958E83AE77
:100800001DD0E751E925EB6FE851EA21EC6F036A4F
:10081000026A016A010E006EEB51ED6F07E0D8909D
:100820000036013602360336ED2FF9D70050E113BA
:100830000150E2130250E3130350E413E52BD8B444
:10084000E62BBED7E86B080EE76FE95F000EEA5BA8
:10085000E66BE56BE65340E1E55107083DE3E75100
:10086000D8B4E807E707959A8C9ADBCA00F0E751FD
:10087000016E04E0D8900032012EFCD700B002D007
:100880008C9C01D08C8C959C00D0959A8C8A00D041
:10089000958E83AE1DD0E751E925EB6FE851EA2133
:1008A000EC6F036A026A016A010E006EEB51ED6F94
:1008B00007E0D8900036013602360336ED2FF9D71F
:1008C0000050E1130150E2130250E3130350E4130C
:1008D000E52BD8B4E62BBED7E86B080EE76FE95FCF
:1008E000000EEA5BE66BE56BE65340E1E551070875
:1008F0003DE3E751D8B4E807E707959A8C9ADCCA3C
:1009000000F0E751016E04E0D8900032012EFCD7D0
:1009100000B002D08C9C01D08C8C959C00D0959A14
:100920008C8A00D0958E83AE1DD0E751E925EB6F00
:10093000E851EA21EC6F036A026A016A010E006E57
:10094000EB51ED6F07E0D8900036013602360336E2
:10095000ED2FF9D70050E1130150E2130250E313D9
:100960000350E413E52BD8B4E62BBED7959A8C8AB6
:1009700000D000D095988C88E1CA00F0E2CA01F05E
:10098000E3CA02F0E4CA03F00001D6EF04F00A0162
:10099000D86BD76BD66BD56BD1CAD9FAD2CADAFA73
:1009A000D3CADBFAD4CADCFA0001BFD603C0D8FA36
:1009B00002C0D7FA01C0D6FA00C0D5FA100E006EF8
:1009C000002EFED70000D5CA00F0D6CA01F0D7CA63
:1009D00002F0D8CA03F0000C0A01C86BC76BC86BE1
:1009E000800EC76FC85100082BE37F0EC75DC96F2B
:1009F000000EC859CA6F660EC925E96E000ECA21DD
:100A0000EA6EEFCFC9FA800EC75DCA6F000EC859F3
:100A1000CB6F660ECA25E96E000ECB21EA6EEFCFD2
:100A2000CAFAC7CAD1FAD26BC9CAD3FACACAD4FAA7
:100A30000001ADDF020E0A01C727000EC823D2D77E
:100A40007E0ED16F110ED26F070ED36F210ED46FB1
:100A500000019DDF100E0A01D16F020ED26F100E41
:100A6000D36F400ED46F000192DF300E0A01D16FB8
:100A7000020ED26F100ED36F400ED46F000187DFCD
:100A8000180E0A01D16FD26B560ED36F060ED46FBB
:100A900000017DDF380E0A01D16FD26B560ED36F85
:100AA000060ED46F000173DF040E0A01D16FD26B02
:100AB000D36B020ED46F00016ADF060E0A01D16FFC
:100AC000D26B030ED36F520ED46F000160DF0C0E99
:100AD0000A01D16FD26BD36B280ED46F000157DFA0
:100AE000120E0A01D16FD26B980ED36F060ED46F1F
:100AF00000014DDF140E0A01D16FD26B0F0ED36FC0
:100B0000D46B000144DF020E0A01D16FD26BD36BAC
:100B1000D46B00013CDF0A01D16BD26BD36BD46B79
:100B2000000135DF240E0A01D16FD26BD36B020EA8
:100B3000D46F00012CDF260E0A01D16FD26B030E99
:100B4000D36FB60ED46F000122DF2C0E0A01D16FD5
:100B5000D26BD36B280ED46F000119DF320E0A015D
:100B6000D16FD26B980ED36F060ED46F00010FDFDA
:100B7000340E0A01D16FD26B0F0ED36FD46B00010C
:100B800006DF220E0A01D16FD26BD36BD46B00014A
:100B9000FEDE200E0A01D16FD26BD36BD46B000145
:100BA000F6DE000C0A0EEA6EC80EE96EEF500EE09B
:100BB000050E016E006A002EFED7012EFBD72E0E09
:100BC000006E002EFED700D0EF2EF2D7000C0A01E7
:100BD0009CCAE9FF9DCAEAFFEFCFA0FA9FCA03F0C3
:100BE0009ECAE9FF9FCAEAFFEF50A05D15E19DCACA
:100BF00003F09CCAE9FF03C0EAFFEF5203E1000ED5
:100C0000016E1FD09DCA03F09C519C2BD8B49D2B24
:100C10009E2BD8B49F2BDCD79DCA03F09CCAE9FF5A
:100C20009DCAEAFFEFCFA0FA9FCA03F09ECAE9FF70
:100C30009FCAEAFFEF50A05D02E2FF0E01D0010E55
:100C4000016E000160EF06F00A018E6B906B8F6BF6
:100C5000200E916F926F936F946F956F966F976F51
:100C6000986F996F9A6F9B6B030E906FEF0E8F6F5B
:100C70008E6B8E5109081BE3036A8E51910FE96E4A
:100C80000A0E0320EA6EF2CF9EFAF29E90CAAAFFE5
:100C90008FCAA9FFA69CA69EA680A8509EBFF28ED2
:100CA000EF6E010E8F27000E90238E2BE2D70A0ED7
:100CB0009D6F910E9C6F9F6B290E9E6F000187D7D1
:100CC000015204E1010E016E04D003D0000E016E4A
:100CD00000D034EF28F00A01946B936B946B936B04
:100CE000945103081CE394CAAAFF93CAA9FFFF0EFC
:100CF000A86EA69CA69EA684F250006EF29E0F01DE
:100D0000550EA76EAA0EA76EA682A6B2FED7A6940F
:100D10000050F2120A01932BD8B4942BE1D70001B2
:100D2000D1EF06F00A01946B936B956B966B946B05
:100D3000200E936F956B95510F0828E3966B965193
:100D40000F0822E39451036E9351932BD8B4942B44
:100D5000976F03C098FA98CAAAFF97CAA9FFA86A12
:100D6000A69CA69EA684F250006EF29E0F01550E20
:100D7000A76EAA0EA76EA682A6B2FED7A6940050B2
:100D8000F2120A01962BDBD7952BD5D7000163EF22
:100D900007F00A018F6B8E6B916B906B926B000169
:100DA0009AD7AA6AA96AA86AA69CA69EA684F250A7
:100DB000006EF29E0F01550EA76EAA0EA76EA682B8
:100DC000A6B2FED7A6940050F212AA6A010EA96E2E
:100DD0000E0EA86EA69CA69EA684F2CF00F0F29EF0
:100DE000550EA76EAA0EA76EA682A6B2FED7A6942F
:100DF0000050F212AA6A020EA96E0A0EA86EA69CF4
:100E0000A69EA684F2CF00F0F29E550EA76EAA0E03
:100E1000A76EA682A6B2FED7A6940050F212AA6AC6
:100E2000030EA96E4F0EA86EA69CA69EA684F2CFB6
:100E300000F0F29E550EA76EAA0EA76EA682A6B26D
:100E4000FED7A6940050F212AA6A040EA96EA86AF0
:100E5000A69CA69EA684F2CF00F0F29E550EA76E29
:100E6000AA0EA76EA682A6B2FED7A6940050F212D2
:100E7000AA6A050EA96E4F0EA86EA69CA69EA68411
:100E8000F2CF00F0F29E550EA76EAA0EA76EA682B4
:100E9000A6B2FED7A6940050F212AA6A060EA96E58
:100EA000A86AA69CA69EA684F2CF00F0F29E550EDC
:100EB000A76EAA0EA76EA682A6B2FED7A694005071
:100EC000F21200012FD7030E0A018F6FEF0E8E6F03
:100ED000926B92510A0827E3036A9251290FE96E37
:100EE000000E0320EA6EEFCF93FA8FCAAAFF8ECAD4
:100EF000A9FF93CAA8FFA69CA69EA684F250006EE6
:100F0000F29E0F01550EA76EAA0EA76EA682A6B27C
:100F1000FED7A6940050F212010E0A018E27000E91
:100F20008F23922BD6D7916B906B926B92510808BE
:100F300043E3036A9251340FE96E000E0320EA6E18
:100F4000EFCF93FA93512F0803E29351390802E24D
:100F5000000E01D0010E01082DE191532BE19051BB
:100F6000050828E3036A9251340FE96E000E03204E
:100F7000EA6EEFCF93FA8FCAAAFF8ECAA9FF93CA6F
:100F8000A8FFA69CA69EA684F250006EF29E0F01BA
:100F9000550EA76EAA0EA76EA682A6B2FED7A6947D
:100FA0000050F2120A01902BD8B4912B010E8E271B
:100FB000000E8F23922BBAD7000139EF28F0F2CF21
:100FC0008EFAF29EAA6AA96AA69CA69EA680A8503E
:100FD0000A018EBFF28E02016E6FF2CF8EFAF29E80
:100FE000AA6A010EA96EA69CA69EA680A8500A0118
:100FF0008EBFF28E02016F6FF2CF8EFAF29EAA6A56
:10100000020EA96EA69CA69EA680A8500A018EBFBD
:10101000F28E0201706FF2CF8EFAF29EAA6A030E70
:10102000A96EA69CA69EA680A8500A018EBFF28E2D
:101030000201716FF2CF8EFAF29EAA6A040EA96EB7
:10104000A69CA69EA680A8500A018EBFF28E020121
:10105000726FF2CF8EFAF29EAA6A050EA96EA69C56
:10106000A69EA680A8500A018EBFF28E0201736F61
:10107000F2CF8EFAF29EAA6A060EA96EA69CA69ED2
:10108000A680A8500A018EBFF28E0201746F010E75
:10109000016E00013BEF28F0006A016A0A01D0519D
:1010A000D890D1B1002600320132D1B300260032EF
:1010B0000132D1B5002600320132D1B7002600320C
:1010C0000132D1B9002600320132D1BB00260032F4
:1010D0000132D1BD002600320132D1BF00260032DC
:1010E000013200018FEF08F00A01CC6BCB6BCA6BA9
:1010F000C96BCD6BC751C7AF03D0000ED880C755A1
:10110000CD6FC82DA7D0C751C7AF03D0000ED88070
:10111000C755CF6FD06F020ED16F0001BDD7015000
:10112000036AAE0FE96E010E0320EA6EECCF03F006
:10113000ED52EFCF00F003C001F0026A036A01AE86
:1011400002D00206030603C0CCFA02C0CBFA01C0EB
:10115000CAFA00C0C9FA0A01C7BF01D00BD0C91F23
:10116000CA1FCB1FCC1FC92BD8B4CA2BD8B4CB2BCA
:10117000D8B4CC2B036ACD51020FE96E020E0320C6
:10118000EA6EEFCFCEFA0C0ED16FD26BD36BCECA14
:10119000D4FA0001C7EC04F0036A0A01CD51170F1D
:1011A000E96E020E0320EA6EEFCFCEFA036ACD514C
:1011B0002C0FE96E020E0320EA6EEFCFCFFA120E6B
:1011C000D16FD26BCECAD3FACFCAD4FA0001C7EC22
:1011D00004F0100E0A01D16F040ED26F100ED36FFF
:1011E000400ED46F0001C7EC04F0036A0A01CD5130
:1011F000410FE96E020E0320EA6EEF38CE6FF00E5B
:10120000CE17180ED16FD26BCECAD3FA040ED46F9C
:101210000001C7EC04F0140E0A01D16FD26B0F0E5F
:10122000D36F020ED46F0001C7EC04F0CBCACEFA24
:10123000CACACFFAC9CAD0FA080E0A01D16FCBCAFE
:10124000D2FACACAD3FAC9CAD4FA0001C7EC04F068
:101250009AD00A01D890CD35036AE60FE96E000EE8
:101260000320EA6EECCF03F0ED52EFCF00F003C0A5
:1012700001F0026A036A01AE02D00206030603C04F
:10128000CCFA02C0CBFA01C0CAFA00C0C9FAC7BF83
:1012900001D00BD0C91FCA1FCB1FCC1FC92BD8B47C
:1012A000CA2BD8B4CB2BD8B4CC2B036ACD514A0F60
:1012B000E96E010E0320EA6EEFCFCEFA2C0ED16F4D
:1012C000D26BD36BCECAD4FA0001C7EC04F0036A28
:1012D0000A01CD51630FE96E010E0320EA6EEFCFD4
:1012E000CEFA036ACD517C0FE96E010E0320EA6E3F
:1012F000EFCFCFFA320ED16FD26BCECAD3FACFCAAC
:10130000D4FA0001C7EC04F0300E0A01D16F040ECC
:10131000D26F100ED36F400ED46F0001C7EC04F0F3
:10132000036A0A01CD51950FE96E010E0320EA6EA2
:10133000EF38CE6FF00ECE17380ED16FD26BCECA0B
:10134000D3FA040ED46F0001C7EC04F0340E0A0186
:10135000D16FD26B0F0ED36F020ED46F0001C7ECAA
:1013600004F0CBCACEFACACACFFAC9CAD0FA280E3C
:101370000A01D16FCBCAD2FACACAD3FAC9CAD4FAFF
:101380000001C7EC04F0000C0A01CA6BC96BC82D40
:101390006DD0C7530CE1060ED16FD26B030ED36F25
:1013A000520ED46F0001C7EC04F01ED00A01D89091
:1013B000C735036AD80FE96E010E0320EA6EECCF41
:1013C00003F0ED52EFCFC9FA03C0CAFACACACBFA8A
:1013D000C9CACCFA060ED16FD26BCACAD3FAC9CA2F
:1013E000D4FA0001C7EC04F0040E0A01D16FD26BED
:1013F000D36B020ED46F0001C7EC04F00C0E0A018F
:10140000D16FD26BD36B280ED46F0001C7EC04F000
:10141000120E0A01D16FD26B980ED36F060ED46FE5
:101420000001C7EC04F0100E0A01D16F040ED26F58
:10143000100ED36F400ED46F0001C7EC04F0180EED
:101440000A01D16FD26B440ED36F040ED46F00012A
:10145000C7EC04F0140E0A01D16FD26B0F0ED36FDC
:10146000D46B0001C7EC04F06CD00A01C7530CE147
:10147000260ED16FD26B030ED36FB60ED46F000160
:10148000C7EC04F01ED00A01D890C735036A180FC4
:10149000E96E010E0320EA6EECCF03F0ED52EFCFC0
:1014A000C9FA03C0CAFACACACBFAC9CACCFA260E0C
:1014B000D16FD26BCACAD3FAC9CAD4FA0001C7EC39
:1014C00004F0240E0A01D16FD26BD36B020ED46FDD
:1014D0000001C7EC04F02C0E0A01D16FD26BD36B64
:1014E000280ED46F0001C7EC04F0320E0A01D16F50
:1014F000D26B980ED36F060ED46F0001C7EC04F0C8
:10150000300E0A01D16F040ED26F100ED36F400E51
:10151000D46F0001C7EC04F0380E0A01D16FD26B12
:10152000440ED36F040ED46F0001C7EC04F0340EE8
:101530000A01D16FD26B0F0ED36FD46B0001C7ECD1
:1015400004F0000C0A01BE6B010EBD6F110EBC6FE2
:10155000700EBB6FC26B010EC16F110EC06F700EAB
:10156000BF6FC66BC56BC46BC36B4A820001ECECEA
:1015700004F0100E006E002EFED7000092988988AD
:10158000220E0A01D16FD26BD36BD46B0001C7EC72
:1015900004F0200E0A01D16FD26BD36BD46B000123
:1015A000C7EC04F00A01C66BC56B020EC46F580E7F
:1015B000C36F0A0EC76FC86B000196DD0A01C26BCC
:1015C000C16BC06BBF6BC2BF0BD0C25329E1C1530B
:1015D00027E1C051020824E303E1BF51570820E38B
:1015E0000A0EC86F0001D2EC05F0230E0A01D16F7C
:1015F000D26BD36BD46B0001C7EC04F003C0C2FA0A
:1016000002C0C1FA01C0C0FA00C0BFFA0A01C1AFEE
:1016100002D0FF0EC213938081B001D001D0D3D786
:10162000C76BC86B000160DD230E0A01D16FD26B5E
:10163000D36BD46B0001C7EC04F003C0C2FA02C044
:10164000C1FA01C0C0FA00C0BFFA0A01C1AF02D09E
:10165000FF0EC213640EC86F0001D2EC05F0938038
:1016600081B016D00C0E0A01C76FC86B00013CDDBB
:10167000938081B007D0640E0A01C86F0001D2ECDC
:1016800005F0F6D7640E0A01C86F0001D2EC05F030
:10169000230E0A01D16FD26BD36BD46B0001C7EC60
:1016A00004F003C0C2FA02C0C1FA01C0C0FA00C00F
:1016B000BFFA0A01C1AF02D0FF0EC213BDCAC7FAFA
:1016C000BCCAC8FABBCAC9FA220ED16FBDCAD2FAC7
:1016D000BCCAD3FABBCAD4FA0001C7EC04F0BDCA35
:1016E000C7FABCCAC8FABBCAC9FA200E0A01D16F30
:1016F000BDCAD2FABCCAD3FABBCAD4FA0001C7EC3D
:1017000004F056C0BEFA55C0BDFA54C0BCFA53C06E
:10171000BBFA56C0C2FA55C0C1FA54C0C0FA53C091
:10172000BFFAEC0E0A01C76FC86B0001DDDC9380C5
:1017300081A03BD0938081A038D0230E0A01D16FC5
:10174000D26BD36BD46B0001C7EC04F003C0C2FAB8
:1017500002C0C1FA01C0C0FA00C0BFFA0A01C1AF9D
:1017600002D0FF0EC213C2BF09D0C2531CE1C15345
:101770001AE1C05318E1BF51000815E34A82280E50
:10178000D16FD26BD36BD46B0001C7EC04F02A0E7F
:101790000A01D16FD26BD36BD46B0001C7EC04F09C
:1017A0009298899828D20001C5D7280E0A01D16FD6
:1017B000D26BD36BD46B0001C7EC04F02A0E0A0184
:1017C000D16FD26BD36BD46B0001C7EC04F0220E47
:1017D0000A01D16FD26BD36BD46B0001C7EC04F05C
:1017E000200E0A01D16FD26BD36BD46B0001C7EC12
:1017F00004F0010E0A01C76FC86B0001C5DD0A01C4
:10180000C26BC16BC06BBF6BBE6BBD6BBC6BBB6B8C
:10181000938081B02DD0010EBB27D8B0BC2BD8B49B
:10182000BD2BD8B4BE2BBCCAC7FABBCAC8FA200E9F
:10183000D16FD26BBCCAD3FABBCAD4FA0001C7ECD1
:1018400004F0230E0A01D16FD26BD36BD46B00016D
:10185000C7EC04F003C0C2FA02C0C1FA01C0C0FA6A
:1018600000C0BFFA0A01C1AF02D0FF0EC213D0D729
:10187000220ED16FD26BD36BD46B0001C7EC04F096
:10188000200E0A01D16FD26BD36BD46B0001C7EC71
:1018900004F092988998120E0A01C76FC86B000174
:1018A00073DD58C0C7FA57C0C8FA200E0A01D16FBD
:1018B000D26B58C0D3FA57C0D4FA0001C7EC04F079
:1018C000020E0A01D16FD26BD36BD46B0001C7EC4F
:1018D00004F00A01D16BD26BD36BD46B0001C7EC5F
:1018E00004F0938281A250D00A0E0A01C76F010E44
:1018F000C86F000174EC08F0938281A23FD0030E00
:101900000A01D16FD26BD36BD46B0001C7EC04F02A
:1019100003C0C2FA02C0C1FA01C0C0FA00C0BFFAD7
:101920000A01C1AF02D0FF0EC213C2BF21D0C25301
:101930000BE1C15309E1000160510A01C05D18E3E8
:1019400003E15F50BF5D14E34A82080ED16FD26B92
:10195000D36BD46B0001C7EC04F00A0E0A01D16FFF
:10196000D26BD36BD46B0001C7EC04F044D10A01F5
:10197000640EC86F0001D2EC05F0BED7640E0A01F8
:10198000C86F0001D2EC05F0E80E5F240A01BB6FBE
:10199000030E000160210A01BC6FBD6BBE6B026AC1
:1019A000036A03C0C2FA02C0C1FA60C0C0FA5FC0D5
:1019B000BFFABDCAC7FABCCAC8FABBCAC9FA020E86
:1019C000D16FBDCAD2FABCCAD3FABBCAD4FA0001DD
:1019D000C7EC04F0BDCAC7FABCCAC8FABBCAC9FA88
:1019E0000A01D16BBDCAD2FABCCAD3FABBCAD4FAB7
:1019F0000001C7EC04F0F20E0A01C76F010EC86FB8
:101A0000000174EC08F0938281B23FD0938281B2DE
:101A10003CD0140E0A01C86F0001D2EC05F0030E91
:101A20000A01D16FD26BD36BD46B0001C7EC04F009
:101A300003C0C2FA02C0C1FA01C0C0FA00C0BFFAB6
:101A40000A01C1AF02D0FF0EC213C2BF09D0C253F8
:101A50001AE1C15318E1C05316E1BF51000813E366
:101A60004A82080ED16FD26BD36BD46B0001C7ECE6
:101A700004F00A0E0A01D16FD26BD36BD46B000154
:101A8000C7EC04F0B8D00001C1D7080E0A01D16F2D
:101A9000D26BD36BD46B0001C7EC04F00A0E0A01C1
:101AA000D16FD26BD36BD46B0001C7EC04F0020E84
:101AB0000A01D16FD26BD36BD46B0001C7EC04F079
:101AC0000A01D16BD26BD36BD46B0001C7EC04F06D
:101AD000010E0A01C76FC86F000156DC0A01C26B14
:101AE000C16BC06BBF6BBE6BBD6BBC6BBB6B9382C2
:101AF00081A24FD0010EBB27D8B0BC2BD8B4BD2BD0
:101B0000D8B4BE2BBCCAC7FABBCAC8FAD16BD26B59
:101B1000BCCAD3FABBCAD4FA0001C7EC04F0030E66
:101B20000A01D16FD26BD36BD46B0001C7EC04F008
:101B300003C0C2FA02C0C1FA01C0C0FA00C0BFFAB5
:101B40000A01C1AF02D0FF0EC213C2BF21D0C253DF
:101B50000BE1C15309E1000160510A01C05D18E3C6
:101B600003E15F50BF5D14E34A82080ED16FD26B70
:101B7000D36BD46B0001C7EC04F00A0E0A01D16FDD
:101B8000D26BD36BD46B0001C7EC04F034D00A01E4
:101B9000AED7020ED16FD26BD36BD46B0001C7EC02
:101BA00004F00A01D16BD26BD36BD46B0001C7EC8C
:101BB00004F00E0E0A01C76F010EC86F0001C4ECDD
:101BC00009F062C0C7FA61C0C8FA0A01D16BD26BD2
:101BD00062C0D3FA61C0D4FA0001C7EC04F0080E69
:101BE0000A01C76FFA0EC86F0001D2EC05F00A01B6
:101BF000C72FF8D74A920001000C0A01916B906B35
:101C00008F6B8E6B00016551030BD8B402D1230E8C
:101C10000A01D16FD26BD36BD46B0001C7EC04F017
:101C200003C069F202C068F201C067F200C066F248
:101C3000020168AF02D0FF0E6913000165A167D0F1
:101C4000BC0E5724006E7F0E5820016E000E5920E6
:101C5000026E000E5A20E8CF91FA02C090FA01C03D
:101C60008FFA00C08EFA0A0191AF04D0020169AF69
:101C70001ED003D0020169BF48D00A019151020170
:101C8000695D43E314E10A0190510201685D3DE39F
:101C90000EE10A018F510201675D37E308E16651E9
:101CA0000A018E5DD8A002D002012FD00201280EB9
:101CB0000A01D16FD26BD36BD46B0001C7EC04F077
:101CC0002A0E0A01D16FD26BD36BD46B0001C7EC23
:101CD00004F0659165930A0E0A01C76FC86B000195
:101CE000C4EC09F090CA92FA8FCA93FA8ECA94FA99
:101CF000200E0A01D16F90CAD2FA8FCAD3FA8ECAC7
:101D0000D4FA0001C7EC04F0020167D0000165A31A
:101D100063D0BC0E575C006E7F0E5858016E000EEB
:101D20005958026E000E5A58E8CF91FA02C090FA44
:101D300001C08FFA00C08EFA020169AF04D00A0117
:101D400091AF1ED003D00A0191BF47D00201695163
:101D50000A01915D42E314E1020168510A01905DBC
:101D60003CE30EE1020167510A018F5D36E308E1B1
:101D70008E510201665DD8A002D00A012ED00A0160
:101D8000280ED16FD26BD36BD46B0001C7EC04F07B
:101D90002A0E0A01D16FD26BD36BD46B0001C7EC52
:101DA00004F0659165930A0E0A01C76FC86B0001C4
:101DB000C4EC09F090CA92FA8FCA93FA8ECA94FAC8
:101DC000200E0A01D16F90CAD2FA8FCAD3FA8ECAF6
:101DD000D4FA0001C7EC04F00A01000165510C0BB4
:101DE00018E1030E0A01D16FD26BD36BD46B0001E3
:101DF000C7EC04F003C06DF202C06CF201C06BF2DC
:101E000000C06AF202016CAF02D0FF0E6D1301D167
:101E1000000165510C0BD8B4CDD0030E0A01D16F6F
:101E2000D26BD36BD46B0001C7EC04F003C06DF22E
:101E300002C06CF201C06BF200C06AF202016CAF2A
:101E400002D0FF0E6D13000165A734D002016DBFF3
:101E500009D06D532DE16C532BE16B5329E16A518D
:101E6000000826E3080E0A01D16FD26BD36BD46B46
:101E70000001C7EC04F00A0E0A01D16FD26BD36BDC
:101E8000D46B0001C7EC04F0659765950A0E0A0152
:101E9000C76F010EC86F0001C4EC09F00A01D16BD5
:101EA000D26BD36B010ED46F0001C7EC04F00201BA
:101EB00065D0000165A561D0010E5F5C006E000E6B
:101EC0006059036E005003C001F0026A036A03C048
:101ED00091FA02C090FA01C08FFA00C08EFA0A018E
:101EE00091AF04D002016DAF1ED003D002016DBFCF
:101EF00045D00A01915102016D5D40E314E10A01F0
:101F0000905102016C5D3AE30EE10A018F5102012A
:101F10006B5D34E308E16A510A018E5DD8A002D0FE
:101F200002012CD00201080E0A01D16FD26BD36BD3
:101F3000D46B0001C7EC04F00A0E0A01D16FD26B1A
:101F4000D36BD46B0001C7EC04F0659765950A0E5E
:101F50000A01C76F010EC86F0001C4EC09F08FCAF7
:101F600092FA8ECA93FA0A01D16BD26B8FCAD3FA56
:101F70008ECAD4FA0001C7EC04F0020100016551D9
:101F8000030B18E1230E0A01D16FD26BD36BD46B14
:101F90000001C7EC04F003C069F202C068F201C09E
:101FA00067F200C066F2020168AF02D0FF0E69134B
:101FB00030D0000165510F0B2CE1230E0A01D16FC7
:101FC000D26BD36BD46B0001C7EC04F003C069F291
:101FD00002C068F201C067F200C066F2020168AF99
:101FE00002D0FF0E6913030E0A01D16FD26BD36BBF
:101FF000D46B0001C7EC04F003C06DF202C06CF2B8
:1020000001C06BF200C06AF202016CAF02D0FF0E99
:102010006D130001000C0A01BC6703D0BD6702D03C
:1020200007D0BD2BBBCAEEFFBC2FFCD7BD2FFAD704
:1020300000015EEF14F07D0E02017725E96E020EBD
:102040007821EA6EEFCFC3FA0A01010E020177256B
:102050000A01C46F000E020178210A01C56FC4CACB
:1020600077F20A01C551030B0201786F7551775D54
:1020700005E17651785D02E10A017F910A01C3CA48
:1020800001F0000161EF10F00A01C06BBF6B7D53DE
:1020900047E07FA145D0BECA03F0BDCAE9FFBECA72
:1020A000EAFFEF50C0533CE1BF5D3AE2BB51BF25B0
:1020B000016EBC51C021036E01C0C1FAC26F0001A4
:1020C000BAD7C2CAEAFFC1CAE9FF01C0EFFF0A01DD
:1020D000BB51BF25E96EBC51C021EA6EEF3C0ED06A
:1020E000BF5302E1C0530AE07D07BDCAE9FFBECA83
:1020F000EAFFBFCAEFFF010E016E14D0BECA03F0A3
:10210000BDCAE9FFBECAEAFFEF50C05306E1BF5D9A
:1021100004E2BF2BD8B4C02B02D0C06BBF6BB7D7C3
:10212000000E016E00016AEF14F07D0E02017925A8
:10213000E96E060E7A21EA6EC0CAEFFF010E79251C
:102140000A01C16F000E02017A210A01C26FC1CAE1
:1021500079F20A01C251030B02017A6F0A017F83EF
:10216000C03D03D07E2B97988E980001000CAA6A80
:10217000A96A6EC2A8FFA69CA69EA684F250006E15
:10218000F29E0F01550EA76EAA0EA76EA682A6B2EA
:10219000FED7A6940050F212AA6A010EA96E6FC271
:1021A000A8FFA69CA69EA684F2CF00F0F29E550E34
:1021B000A76EAA0EA76EA682A6B2FED7A69400505E
:1021C000F212AA6A020EA96E70C2A8FFA69CA69E71
:1021D000A684F2CF00F0F29E550EA76EAA0EA76E4F
:1021E000A682A6B2FED7A6940050F212AA6A030EE7
:1021F000A96E71C2A8FFA69CA69EA684F2CF00F08D
:10220000F29E550EA76EAA0EA76EA682A6B2FED7A4
:10221000A6940050F212AA6A040EA96E72C2A8FF18
:10222000A69CA69EA684F2CF00F0F29E550EA76E45
:10223000AA0EA76EA682A6B2FED7A6940050F212EE
:10224000AA6A050EA96E73C2A8FFA69CA69EA684C4
:10225000F2CF00F0F29E550EA76EAA0EA76EA682D0
:10226000A6B2FED7A6940050F212AA6A060EA96E74
:1022700074C2A8FFA69CA69EA684F2CF00F0F29E90
:10228000550EA76EAA0EA76EA682A6B2FED7A6947A
:102290000050F2120001000C0A01BD6BBC6BBE6B5A
:1022A000BB51100803E2000E016EFDD0BB51100DB2
:1022B000F350BD6BBC6F200EBC27000EBD23FF0E7C
:1022C000BE6FBDCAAAFFBCCAA9FFBECAA8FFA69C12
:1022D000A69EA684F250006EF29E0F01550EA76EC8
:1022E000AA0EA76EA682A6B2FED7A6940050F2123E
:1022F0000A01BC2BD8B4BD2BBDCAAAFFBCCAA9FF1A
:10230000BECAA8FFA69CA69EA684F250006EF29EAE
:102310000F01550EA76EAA0EA76EA682A6B2FED713
:10232000A6940050F2120A01BC2BD8B4BD2BBDCA32
:10233000AAFFBCCAA9FFBECAA8FFA69CA69EA684E7
:10234000F250006EF29E0F01550EA76EAA0EA76EF8
:10235000A682A6B2FED7A6940050F2120A01BC2BA8
:10236000D8B4BD2BBDCAAAFFBCCAA9FFBECAA8FF6C
:10237000A69CA69EA684F250006EF29E0F01550EFA
:10238000A76EAA0EA76EA682A6B2FED7A69400508C
:10239000F2120A01BC2BD8B4BD2BBDCAAAFFBCCA1D
:1023A000A9FFBECAA8FFA69CA69EA684F250006EF6
:1023B000F29E0F01550EA76EAA0EA76EA682A6B2B8
:1023C000FED7A6940050F2120A01BC2BD8B4BD2B44
:1023D000BDCAAAFFBCCAA9FFBECAA8FFA69CA69EEA
:1023E000A684F250006EF29E0F01550EA76EAA0E43
:1023F000A76EA682A6B2FED7A6940050F2120A01DA
:10240000BC2BD8B4BD2BBDCAAAFFBCCAA9FFBECA8B
:10241000A8FFA69CA69EA684F250006EF29E0F0115
:10242000550EA76EAA0EA76EA682A6B2FED7A694D8
:102430000050F2120A01BC2BD8B4BD2BBDCAAAFFB2
:10244000BCCAA9FFBECAA8FFA69CA69EA684F2503D
:10245000006EF29E0F01550EA76EAA0EA76EA68201
:10246000A6B2FED7A6940050F2120A01BC2BD8B433
:10247000BD2BBDCAAAFFBCCAA9FFBECAA8FFA69CA5
:10248000A69EA684F250006EF29E0F01550EA76E16
:10249000AA0EA76EA682A6B2FED7A6940050F2128C
:1024A000010E016E0A01000183EF1CF00A01BD6BF1
:1024B000BC6BBE6BBB51100803E2000E016E0FD166
:1024C000BB51100DF350BD6BBC6F200EBC27000E2E
:1024D000BD23BDCAAAFFBCCAA9FFBBCAA8FFA69C50
:1024E000A69EA684F250006EF29E0F01550EA76EB6
:1024F000AA0EA76EA682A6B2FED7A6940050F2122C
:102500000A01BC2BD8B4BD2B4EC0BEFABDCAAAFF6F
:10251000BCCAA9FFBECAA8FFA69CA69EA684F2506C
:10252000006EF29E0F01550EA76EAA0EA76EA68230
:10253000A6B2FED7A6940050F2120A01BC2BD8B462
:10254000BD2B4DC0BEFABDCAAAFFBCCAA9FFBECAF8
:10255000A8FFA69CA69EA684F250006EF29E0F01D4
:10256000550EA76EAA0EA76EA682A6B2FED7A69497
:102570000050F2120A01BC2BD8B4BD2B4CC0BEFADD
:10258000BDCAAAFFBCCAA9FFBECAA8FFA69CA69E38
:10259000A684F250006EF29E0F01550EA76EAA0E91
:1025A000A76EA682A6B2FED7A6940050F2120A0128
:1025B000BC2BD8B4BD2B4BC0BEFABDCAAAFFBCCA47
:1025C000A9FFBECAA8FFA69CA69EA684F250006ED4
:1025D000F29E0F01550EA76EAA0EA76EA682A6B296
:1025E000FED7A6940050F2120A01BC2BD8B4BD2B22
:1025F0006DC2BEFA0A01BDCAAAFFBCCAA9FFBECA03
:10260000A8FFA69CA69EA684F250006EF29E0F0123
:10261000550EA76EAA0EA76EA682A6B2FED7A694E6
:102620000050F2120A01BC2BD8B4BD2B6CC2BEFA0A
:102630000A01BDCAAAFFBCCAA9FFBECAA8FFA69CC0
:10264000A69EA684F250006EF29E0F01550EA76E54
:10265000AA0EA76EA682A6B2FED7A6940050F212CA
:102660000A01BC2BD8B4BD2B6BC2BEFA0A01BDCA8D
:10267000AAFFBCCAA9FFBECAA8FFA69CA69EA684A4
:10268000F250006EF29E0F01550EA76EAA0EA76EB5
:10269000A682A6B2FED7A6940050F2120A01BC2B65
:1026A000D8B4BD2B6AC2BEFA0A01BDCAAAFFBCCA11
:1026B000A9FFBECAA8FFA69CA69EA684F250006EE3
:1026C000F29E0F01550EA76EAA0EA76EA682A6B2A5
:1026D000FED7A6940050F212010E016E0A0100010D
:1026E00066EF1DF00A01BD6BBC6BBE6BBB511008E1
:1026F00003E2000E016EBAD0BB51100DF350BD6B5A
:10270000BC6F200EBC27000EBD23F2CFC4FAF29E90
:10271000BDCAAAFFBCCAA9FFA69CA69EA680A850B7
:10272000C4BFF28EBE6FBB51BE5DD8A49CD0BC2B83
:10273000D8B4BD2BF2CFC4FAF29EBDCAAAFFBCCA60
:10274000A9FFA69CA69EA680A850C4BFF28EC26F09
:10275000BC2BD8B4BD2BF2CFC4FAF29EBDCAAAFFDF
:10276000BCCAA9FFA69CA69EA680A850C4BFF28E94
:10277000C16FBC2BD8B4BD2BF2CFC4FAF29EBDCA38
:10278000AAFFBCCAA9FFA69CA69EA680A850C4BF4B
:10279000F28EC06FBC2BD8B4BD2BF2CFC4FAF29E20
:1027A000BDCAAAFFBCCAA9FFA69CA69EA680A85027
:1027B000C4BFF28EBF6FC2CA4EF0C1CA4DF0C0CACC
:1027C0004CF0BFCA4BF0BC2BD8B4BD2BF2CFC4FA2F
:1027D000F29EBDCAAAFFBCCAA9FFA69CA69EA6805F
:1027E000A850C4BFF28EC26FBC2BD8B4BD2BF2CFA1
:1027F000C4FAF29EBDCAAAFFBCCAA9FFA69CA69EA7
:10280000A680A850C4BFF28EC16FBC2BD8B4BD2B1C
:10281000F2CFC4FAF29EBDCAAAFFBCCAA9FFA69C09
:10282000A69EA680A850C4BFF28EC06FBC2BD8B4A1
:10283000BD2BF2CFC4FAF29EBDCAAAFFBCCAA9FF43
:10284000A69CA69EA680A850C4BFF28EBF6FC2CA27
:1028500052F0C1CA51F0C0CA50F0BFCA4FF0010EC9
:10286000016E04D003D0000E016E00D00001F1EF24
:102870001DF00A01916B906B8F6B8E6B956B946B57
:10288000936B926B996B986B976B966B9D6B9C6B34
:102890009B6B9A6BB76B190EB86FB96BBA917D537E
:1028A000D8B49EEF20F00A0EEA6E9E0EE96EBB6B66
:1028B000BD6B190EBC6F00010BEF10F00A0E0A0180
:1028C000BC6F9E0EBB6F0A0EBE6FB80EBD6F0001CF
:1028D00044EF10F0012C9CEF20F00A019E517F0B79
:1028E000B76FB751000A000154E0010A6AE0050A17
:1028F000D8B411D1010AD8B423D20D0AD8B458D211
:102900000A0AD8B4BAD2010AD8B409EF19F0050AF4
:10291000D8B4B1EF1AF0010AD8B4C9EF1AF0090A15
:10292000D8B4E1EF1AF0020AD8B40EEF1CF01D0A79
:10293000D8B443EF1CF0010AD8B463EF1CF0190AB5
:10294000D8B47FEF1CF0030AD8B4B8EF1CF0010A2A
:10295000D8B49AEF1DF0180AD8B4BFEF1EF0070ADA
:10296000D8B4E1EF1EF01B0AD8B401EF1FF0020A41
:10297000D8B41CEF1FF01F0AD8B43BEF1FF0070AB2
:10298000D8B486EF1FF0030AD8B4FDEF1FF080EF34
:1029900020F0400E0A01C06F000195EC10F00A0112
:1029A000C06B000195EC10F00A01C06B000195ECC2
:1029B00010F0FF0E0A01C06F000195EC10F09CEFC3
:1029C00020F04AA202D0ADEF20F00A01A151030B82
:1029D000030838E1A251030B030834E1280ED16F3C
:1029E000D26BD36BD46B0001C7EC04F0080E0A0164
:1029F000D16FD26BD36BD46B0001C7EC04F0020132
:102A00006EB112D02A0E0A01D16FD26BD36BD46B88
:102A10000001C7EC04F00A0E0A01D16FD26BD36B30
:102A2000D46B0001C7EC04F0030E0A018A6F846FB7
:102A30008B6F856F00016591659365956597ADEF27
:102A400020F00A01A151030B030821E1280ED16FE8
:102A5000D26BD36BD46B0001C7EC04F002016EB1F2
:102A600009D02A0E0A01D16FD26BD36BD46B00014F
:102A7000C7EC04F00A018A51A15D08E0030E846FDF
:102A800084CA8AFA0001659165930A0124D0A25193
:102A9000030B030820E1080ED16FD26BD36BD46B0C
:102AA0000001C7EC04F002016EB109D00A0E0A0160
:102AB000D16FD26BD36BD46B0001C7EC04F00A0169
:102AC0008B51A25D08E0030E856F85CA8BFA000169
:102AD000659565970A01B96BB951040819E3036A52
:102AE000B951810F016E0A0E032203C0BCFA036ABA
:102AF000B9519E0FE96E0A0E0320EA6EEFCFBDFAC0
:102B0000BCCAEAFF01C0E9FFBDCAEFFFB92BE4D799
:102B100000019CEF20F04AA21AD0440E0A01C06FB7
:102B2000000195EC10F0080E0A01C06F000195EC51
:102B300010F0030E0A01C06F000195EC10F0FF0EBB
:102B40000A01C06F000195EC10F0ADEF20F02752A4
:102B5000D8A4DED0230E0A01D16FD26BD36BD46B15
:102B60000001C7EC04F003C091FA02C090FA01C062
:102B70008FFA00C08EFA0A0190AF02D0FF0E9113B7
:102B800057508E5D09E158508F5D06E15950905DB8
:102B900003E15A50915D19E06FC2C7FAC86B00019A
:102BA000C4EC09F059C0BBFA58C0BCFA57C0BDFA12
:102BB000200E0A01D16F59C0D2FA58C0D3FA57C0BB
:102BC000D4FA0001C7EC04F00A01030ED16FD26BF6
:102BD000D36BD46B0001C7EC04F003C095FA02C0BC
:102BE00094FA01C093FA00C092FA0A0194AF02D09D
:102BF000FF0E9513000161510A01925D09E1000188
:102C000062510A01935D04E1945302E1955316E089
:102C100070C2C7FA010EC86F0001C4EC09F062C0AF
:102C2000BBFA61C0BCFA0A01D16BD26B62C0D3FAA5
:102C300061C0D4FA0001C7EC04F00A01BA91BAB13C
:102C400067D057508E5D19E158508F5D16E159508D
:102C5000905D13E15A50915D10E1000161510A014C
:102C6000925D0BE1000162510A01935D06E194530C
:102C700004E1955302E1BA814AD0640EC86F0001A5
:102C8000D2EC05F057500A018E5D09E158508F5D76
:102C900006E15950905D03E15A50915D15E0230E15
:102CA000D16FD26BD36BD46B0001C7EC04F003C0BF
:102CB00091FA02C090FA01C08FFA00C08EFA0A01A0
:102CC00090AF02D0FF0E9113000161510A01925D95
:102CD00009E1000162510A01935D04E1945302E1AC
:102CE000955315E0030ED16FD26BD36BD46B0001FB
:102CF000C7EC04F003C095FA02C094FA01C093FA3D
:102D000000C092FA0A0194AF02D0FF0E951397D734
:102D1000440E0A01C06F000195EC10F00A01C06B6F
:102D2000000195EC10F00A01C06B000195EC10F069
:102D3000FF0E0A01C06F000195EC10F09CEF20F02F
:102D4000275202E1A2EC0AF04AA21AD0450E0A016B
:102D5000C06F000195EC10F0080E0A01C06F000171
:102D600095EC10F0030E0A01C06F000195EC10F015
:102D7000FF0E0A01C06F000195EC10F0ADEF20F0DE
:102D8000450E0A01C06F000195EC10F00A01C06BFE
:102D9000000195EC10F00A01C06B000195EC10F0F9
:102DA000FF0E0A01C06F000195EC10F09CEF20F0BF
:102DB0004AA21AD0480E0A01C06F000195EC10F02B
:102DC000080E0A01C06F000195EC10F0030E0A0115
:102DD000C06F000195EC10F0FF0E0A01C06F0001FA
:102DE00095EC10F0ADEF20F027522FE16FC2C7FA3B
:102DF0000A01C86B0001C4EC09F070C2C7FA010EE9
:102E00000A01C86F0001C4EC09F05DC0BBFA5CC0E8
:102E1000BCFA5BC0BDFA200E0A01D16F5DC0D2FAC8
:102E20005CC0D3FA5BC0D4FA0001C7EC04F064C004
:102E3000BBFA63C0BCFA0A01D16BD26B64C0D3FA8F
:102E400063C0D4FA0001C7EC04F0480E0A01C06F59
:102E5000000195EC10F00A01C06B000195EC10F038
:102E60000A01C06B000195EC10F0FF0E0A01C06F63
:102E7000000195EC10F09CEF20F04AA21AD0420E0F
:102E80000A01C06F000195EC10F0080E0A01C06F36
:102E9000000195EC10F0030E0A01C06F000195ECE3
:102EA00010F0FF0E0A01C06F000195EC10F0ADEFBD
:102EB00020F02752D8A493D10A01B8510B08D8A406
:102EC00076D1A139BC6FF00EBC17A2510F0BBC1309
:102ED000A339BE6FF00EBE17A4510F0BBE13026ACA
:102EE000036A03C099FA02C098FABCCA97FABECA2C
:102EF00096FA97AF1CD0FF0E9813991399AF16D07E
:102F00009951FF0813E30BE19851FF080FE307E124
:102F1000975180080BE303E19651430807E3FF0E46
:102F2000996F986F800E976F440E966F14D099BF6B
:102F300012D099530AE1985308E197517E080BE2A9
:102F4000FF0A03E19651BC0806E2996B986B7F0E6D
:102F5000976FBC0E966F965157248E6F97515820DD
:102F60008F6F98515920906F99515A20916FA539C0
:102F7000BC6FF00EBC17A6510F0BBC13A739BE6F68
:102F8000F00EBE17A8510F0BBE13026A036A03C0EE
:102F90009DFA02C09CFABCCA9BFABECA9AFA9BAFC1
:102FA0001CD0FF0E9C139D139DAF16D09D51FF08A2
:102FB00013E30BE19C51FF080FE307E19B51E80885
:102FC0000BE303E19A518F0807E3FF0E9D6F9C6F9F
:102FD000E80E9B6F900E9A6F14D09DBF12D09D5338
:102FE0000AE19C5308E19B514B080BE2FF0A03E105
:102FF0009A512C0806E29D6B9C6B4C0E9B6F2C0E1D
:103000009A6F9F5303E1010E9F6F05D09F511808DF
:1030100002E2180E9F6FA05303E1010EA06F05D0CE
:10302000A051140802E2140EA06F000161510A01C0
:103030009A25926F000162510A019B21936F000E45
:103040009C21946F000E9D21956F9FCAC7FAC86B93
:103050000001C4EC09F0A0CAC7FA010E0A01C86F4A
:103060000001C4EC09F090CABBFA8FCABCFA8ECA40
:10307000BDFA200E0A01D16F90CAD2FA8FCAD3FAD4
:103080008ECAD4FA0001C7EC04F094CABBFA93CA02
:10309000BCFA92CABDFA0A01D16B94CAD2FA93CA99
:1030A000D3FA92CAD4FA0001C7EC04F00A01BA912B
:1030B000320EC86F0001D2EC05F0790E0A01996F4B
:1030C000990E986F976F966F790E9D6F990E9C6F02
:1030D0009B6F9A6FBAB152D08E51965D15E18F51A8
:1030E000975D12E19051985D0FE19151995D0CE16E
:1030F00092519A5D09E193519B5D06E194519C5D6B
:1031000003E195519D5D37E0230ED16FD26BD36BF8
:10311000D46B0001C7EC04F003C099FA02C098FA1E
:1031200001C097FA00C096FA0A0198AF02D0FF0ECC
:103130009913320EC86F0001D2EC05F0030E0A019C
:10314000D16FD26BD36BD46B0001C7EC04F003C01A
:103150009DFA02C09CFA01C09BFA00C09AFA0A01CB
:103160009CAF02D0FF0E9D13320EC86F0001D2EC4F
:1031700005F002D00A01BA810A01ACD7420EC06F35
:10318000000195EC10F00A01C06B000195EC10F005
:103190000A01C06B000195EC10F0FF0E0A01C06F30
:1031A000000195EC10F0ADEF20F018D00A01420EAE
:1031B000C06F000195EC10F0080E0A01C06F00010D
:1031C00095EC10F0010E0A01C06F000195EC10F0B3
:1031D000FF0E0A01C06F000195EC10F018D0420EEE
:1031E0000A01C06F000195EC10F00A01C06B0001EC
:1031F00095EC10F00A01C06B000195EC10F0FF0E89
:103200000A01C06F000195EC10F0ADEF20F09CEFCB
:1032100020F04AA21AD0430E0A01C06F000195ECBB
:1032200010F0080E0A01C06F000195EC10F0030EBB
:103230000A01C06F000195EC10F0FF0E0A01C06F8B
:10324000000195EC10F0ADEF20F02752D8A46FD11B
:103250000A01B8510B08D8A452D1230ED16FD26BFA
:10326000D36BD46B0001C7EC04F003C091FA02C029
:1032700090FA01C08FFA00C08EFA0A0190AF02D016
:10328000FF0E9113030ED16FD26BD36BD46B000181
:10329000C7EC04F003C095FA02C094FA01C093FA97
:1032A00000C092FA0A0194AF02D0FF0E9513A13923
:1032B000BC6FF00EBC17A2510F0BBC13A339BE6F2D
:1032C000F00EBE17A4510F0BBE13026A036A03C0AF
:1032D00099FA02C098FABCCA97FABECA96FA97AF92
:1032E00003D0FF0E98139913A539BC6FF00EBC17CD
:1032F000A6510F0BBC13A739BE6FF00EBE17A85115
:103300000F0BBE13026A036A03C09DFA02C09CFA47
:10331000BCCA9BFABECA9AFA9BAF03D0FF0E9C139D
:103320009D1396518E2797518F2398519023995131
:103330009123BC0E5724006E7F0E5820016E000EA4
:103340005920026E000E5A20036E91BF22D0035006
:10335000915D1FE30BE10250905D1BE307E101501B
:103360008F5D17E303E18E51005C13E2BC0E57241E
:10337000006E7F0E5820016E000E5920026E000E66
:103380005A20916F02C090FA01C08FFA00C08EFAE5
:103390002FD0BC0E575C006E7F0E5858016E000E89
:1033A0005958026E000E5A58036E91BF0FD09151BA
:1033B000035C1EE30BE19051025C1AE307E18F51BD
:1033C000015C16E303E100508E5D12E2BC0E575C17
:1033D000006E7F0E5858016E000E5958026E000E96
:1033E0005A58916F02C090FA01C08FFA00C08EFA4D
:1033F0009A5192279B5193239C5194239D5195233D
:1034000095BF18D095530BE1945309E10001605129
:103410000A01935D0FE303E192515F5C0BE2026AE4
:10342000036A03C095FA02C094FA60C093FA5FC0C1
:1034300092FA07D095BF01D004D0956B946B936B33
:10344000926B9F5303E1010E9F6F05D09F511808A7
:1034500002E2180E9F6FA05303E1010EA06F05D08A
:10346000A051140802E2140EA06F9FCAC7FAC86BDD
:103470000001C4EC09F0A0CAC7FA010E0A01C86F26
:103480000001C4EC09F090CABBFA8FCABCFA8ECA1C
:10349000BDFA200E0A01D16F90CAD2FA8FCAD3FAB0
:1034A0008ECAD4FA0001C7EC04F094CABBFA93CADE
:1034B000BCFA92CABDFA0A01D16B94CAD2FA93CA75
:1034C000D3FA92CAD4FA0001C7EC04F0430E0A0101
:1034D000C06F000195EC10F00A01C06B000195EC83
:1034E00010F00A01C06B000195EC10F0FF0E0A010C
:1034F000C06F000195EC10F0ADEF20F00A01430E13
:10350000C06F000195EC10F0080E0A01C06F0001B9
:1035100095EC10F0010E0A01C06F000195EC10F05F
:10352000FF0E0A01C06F000195EC10F018D0430E99
:103530000A01C06F000195EC10F00A01C06B000198
:1035400095EC10F00A01C06B000195EC10F0FF0E35
:103550000A01C06F000195EC10F0ADEF20F09CEF78
:1035600020F0460E0A01C06F000195EC10F00A0130
:10357000C06B000195EC10F00A01C06B000195ECE6
:1035800010F0FF0E0A01C06F000195EC10F09CEFE7
:1035900020F0470E0A01C06F000195EC10F00A01FF
:1035A000C06B000195EC10F00A01C06B000195ECB6
:1035B00010F0FF0E0A01C06F000195EC10F09CEFB7
:1035C00020F04AB259D057500201665D0A018E6F51
:1035D0005850020167590A018F6F5950020168590A
:1035E0000A01906F5A50020169590A01916F91BF07
:1035F00013D091530AE1905308E18F517E080CE2F9
:10360000FF0A03E18E51BC0807E2916B906B7F0EBD
:103610008F6FBC0E8E6F18D091AF16D09151FF08EE
:1036200013E30BE19051FF080FE307E18F5180088E
:103630000BE303E18E51430807E3FF0E916F906F98
:10364000800E8F6F440E8E6F0001615102016A5D22
:103650000A01926F0001625102016B590A01936FD6
:10366000000E02016C590A01946F000E02016D599F
:103670000A01956F0AD000010A01916B906B8F6B64
:103680008E6B956B946B936B926B4E0EC06F0001BB
:1036900095EC10F00A01C06B000195EC10F00A01E6
:1036A000C06B000195EC10F00A01BF6B9131BE6F49
:1036B0009031BD6F8F31BC6FBE33BD33BC33BE3371
:1036C000BD33BC33BE33BD33BC330F0EBE17BC1786
:1036D000BD6BBE6BBF6BBCCAC0FA000195EC10F0AD
:1036E0008FCABCFA90CABDFA91CABEFA0A01BF6B72
:1036F0000F0EBC17BD6BBE6BBF6BBCCAC0FA00011E
:1037000095EC10F00A019131BF6F9031BE6F8F318F
:10371000BD6F8E31BC6FBF33BE33BD33BC33BF33DF
:10372000BE33BD33BC33BF33BE33BD33BC330F0EEA
:10373000BF17BC17BD6BBE6BBF6BBCCAC0FA000124
:1037400095EC10F00A018E510F0BBB6FBC6BBD6B7B
:10375000BE6BC06F000195EC10F00A01BF6B953194
:10376000BE6F9431BD6F9331BC6FBE33BD33BC337C
:10377000BE33BD33BC33BE33BD33BC330F0EBE17B7
:10378000BC17BD6BBE6BBF6BBCCAC0FA000195EC29
:1037900010F093CABCFA94CABDFA95CABEFA0A01DF
:1037A000BF6B0F0EBC17BD6BBE6BBF6BBCCAC0FA44
:1037B000000195EC10F00A019531BF6F9431BE6F96
:1037C0009331BD6F9231BC6FBF33BE33BD33BC3359
:1037D000BF33BE33BD33BC33BF33BE33BD33BC3365
:1037E0000F0EBF17BC17BD6BBE6BBF6BBCCAC0FA58
:1037F000000195EC10F00A0192510F0BBB6FBC6BEE
:10380000BD6BBE6BC06F000195EC10F0FF0E0A019E
:10381000C06F000195EC10F09CEF20F00A019F5161
:10382000000806E29F51180803E39FCA6FF204D014
:103830000E0E02016F6F0A019F51000806E29F51B0
:10384000140803E39FCA70F203D00A0E0201706FDE
:103850000001B7EC10F04C0E0A01C06F000195ECAE
:1038600010F00A01C06B000195EC10F00A01C06B6A
:10387000000195EC10F0FF0E0A01C06F000195ECFD
:1038800010F09CEF20F0510E0A01C06F000195EC82
:1038900010F00A01C06B000195EC10F00A01C06B3A
:1038A000000195EC10F06FC2C0FA95EC10F070C2F8
:1038B000C0FA95EC10F0FF0E0A01C06F000195EC04
:1038C00010F09CEF20F0500E0A01C06F000195EC43
:1038D00010F00A01C06B000195EC10F00A01C06BFA
:1038E000000195EC10F049C0C0FA95EC10F0FF0E05
:1038F0000A01C06F000195EC10F09CEF20F09FCA08
:10390000BBFA4CEF11F0012C19D09FCA49F0490EB7
:103910000A01C06F000195EC10F00A01C06B0001B4
:1039200095EC10F00A01C06B000195EC10F0FF0E51
:103930000A01C06F000195EC10F018D0490E0A0181
:10394000C06F000195EC10F0080E0A01C06F000175
:1039500095EC10F0010E0A01C06F000195EC10F01B
:10396000FF0E0A01C06F000195EC10F09CEF20F0F3
:103970004AA21AD04A0E0A01C06F000195EC10F05D
:10398000080E0A01C06F000195EC10F0030E0A0149
:10399000C06F000195EC10F0FF0E0A01C06F00012E
:1039A00095EC10F0ADEF20F065510F0B35E0280ECF
:1039B0000A01D16FD26BD36BD46B0001C7EC04F05A
:1039C000080E0A01D16FD26BD36BD46B0001C7EC28
:1039D00004F02A0E0A01D16FD26BD36BD46B0001B5
:1039E000C7EC04F00A0E0A01D16FD26BD36BD46B13
:1039F0000001C7EC04F0030E0A018A6F846F8B6F1D
:103A0000856F000165916593659565970A0E0A01BA
:103A1000C86F0001D2EC05F069C24EF068C24DF0EB
:103A200067C24CF066C24BF0BC0E5724006E7F0E8E
:103A30005820016E000E5920026E000E5A20036EAF
:103A40004E5C19E30BE102504D5C15E307E10150B8
:103A50004C5C11E303E14B50005C0DE2BC0E5724BB
:103A60004B6E7F0E58204C6E000E59204D6E000E8E
:103A70005A204E6E27D0BC0E575C006E7F0E5858F1
:103A8000016E000E5958026E000E5A58036E4E50C9
:103A9000035C18E30BE14D50025C14E307E14C506A
:103AA000015C10E303E100504B5C0CE2BC0E575C80
:103AB0004B6E7F0E58584C6E000E59584D6E000ECE
:103AC0005A584E6E9FCABBFA56EF12F0012C19D00D
:103AD0009FCA49F04A0E0A01C06F000195EC10F030
:103AE0000A01C06B000195EC10F00A01C06B0001E7
:103AF00095EC10F0FF0E0A01C06F000195EC10F07C
:103B000018D04A0E0A01C06F000195EC10F0080EA3
:103B10000A01C06F000195EC10F0010E0A01C06FA0
:103B2000000195EC10F0FF0E0A01C06F000195EC4A
:103B300010F002D34AA219D04B0E0A01C06F000147
:103B400095EC10F0080E0A01C06F000195EC10F022
:103B5000030E0A01C06F000195EC10F0FF0E0A0180
:103B6000C06F000195EC10F0F8D265510F0B35E0F5
:103B7000280E0A01D16FD26BD36BD46B0001C7EC56
:103B800004F0080E0A01D16FD26BD36BD46B000125
:103B9000C7EC04F02A0E0A01D16FD26BD36BD46B41
:103BA0000001C7EC04F00A0E0A01D16FD26BD36B8F
:103BB000D46B0001C7EC04F0030E0A018A6F846F16
:103BC0008B6F856F000165916593659565970A0E0A
:103BD0000A01C86F0001D2EC05F09FCABBFA72EF70
:103BE00013F0012CB3D06FC2C7FA0A01C86B0001F1
:103BF000C4EC09F070C2C7FA010E0A01C86F0001D7
:103C0000C4EC09F04DC0BBFA4CC0BCFA4BC0BDFAC5
:103C1000200E0A01D16F4DC0D2FA4CC0D3FA4BC06E
:103C2000D4FA0001C7EC04F051C0BBFA50C0BCFA92
:103C30004FC0BDFA0A01D16B51C0D2FA50C0D3FABD
:103C40004FC0D4FA0001C7EC04F09FCA49F00A0142
:103C5000BA91320EC86F0001D2EC05F0790E0A015C
:103C6000996F990E986F976F966F790E9D6F990E59
:103C70009C6F9B6F9A6FBAB152D04B50965D15E115
:103C80004C50975D12E14D50985D0FE14E50995D9B
:103C90000CE14F509A5D09E150509B5D06E1515097
:103CA0009C5D03E152509D5D37E0230ED16FD26BD6
:103CB000D36BD46B0001C7EC04F003C099FA02C0C7
:103CC00098FA01C097FA00C096FA0A0198AF02D09C
:103CD000FF0E9913320EC86F0001D2EC05F0030EEF
:103CE0000A01D16FD26BD36BD46B0001C7EC04F027
:103CF00003C09DFA02C09CFA01C09BFA00C09AFA68
:103D00000A019CAF02D0FF0E9D13320EC86F000156
:103D1000D2EC05F002D00A01BA810A01ACD74B0EF1
:103D2000C06F000195EC10F00A01C06B000195EC2A
:103D300010F00A01C06B000195EC10F0FF0E0A01B3
:103D4000C06F000195EC10F0F7D118D04B0E0A01AE
:103D5000C06F000195EC10F0080E0A01C06F000161
:103D600095EC10F0010E0A01C06F000195EC10F007
:103D7000FF0E0A01C06F000195EC10F0DDD10A01C1
:103D8000A0A103D002016E8102D002016E91000158
:103D9000B7EC10F0530E0A01C06F000195EC10F063
:103DA0000A01C06B000195EC10F00A01C06B000124
:103DB00095EC10F0FF0E0A01C06F000195EC10F0B9
:103DC000BBD1540E0A01C06F000195EC10F00A013E
:103DD000C06B000195EC10F00A01C06B000195EC7E
:103DE00010F00A01C06B000195EC10F06EC2C0FA31
:103DF00095EC10F0FF0E0A01C06F000195EC10F079
:103E00009BD14F0E0A01C06F000195EC10F00A0122
:103E1000C06B000195EC10F00A01C06B000195EC3D
:103E200010F065C0C0FA95EC10F0FF0E0A01C06FEB
:103E3000000195EC10F080D14D0E0A01C06F000119
:103E400095EC10F00A01C06B000195EC10F00A012E
:103E5000C06B000195EC10F05AC2C0FA95EC10F05E
:103E60005BC2C0FA95EC10F0FF0E0A01C06F0001B2
:103E700095EC10F061D1520E0A01C06F000195EC73
:103E800010F00A01C06B000195EC10F00A01C06B44
:103E9000000195EC10F035C0C0FA95EC10F036C07A
:103EA000C0FA95EC10F038C0C0FA95EC10F039C0AB
:103EB000C0FA95EC10F03BC0C0FA95EC10F03CC095
:103EC000C0FA95EC10F03FC0C0FA95EC10F040C07D
:103ED000C0FA95EC10F042C0C0FA95EC10F043C067
:103EE000C0FA95EC10F044C0C0FA95EC10F046C052
:103EF000C0FA95EC10F047C0C0FA95EC10F0FF0E38
:103F00000A01C06F000195EC10F016D14AA219D039
:103F1000550E0A01C06F000195EC10F0080E0A0161
:103F2000C06F000195EC10F0030E0A01C06F000194
:103F300095EC10F0FF0E0A01C06F000195EC10F037
:103F40000CD10A019F51020808E1246A236A266AFB
:103F5000256A276A020E286E3AD0286A226A216AE8
:103F6000206A1F6A2750020832E2275006082FE213
:103F7000280ED16FD26BD36BD46B0001C7EC04F069
:103F8000080E0A01D16FD26BD36BD46B0001C7EC62
:103F900004F02A0E0A01D16FD26BD36BD46B0001EF
:103FA000C7EC04F00A0E0A01D16FD26BD36BD46B4D
:103FB0000001C7EC04F0030E0A018A6F846F8B6F57
:103FC000856F000165916593659565970A01550EAA
:103FD000C06F000195EC10F00A01C06B000195EC78
:103FE00010F00A01C06B000195EC10F0FF0E0A0101
:103FF000C06F000195EC10F09FD0560E0A01C06F03
:10400000000195EC10F00A01C06B000195EC10F076
:104010000A01C06B000195EC10F024380A01BB6F57
:10402000BC6B0F0EBB17BB17BC6BBBCAC0FA000141
:1040300095EC10F024C0BBFA0A01BC6B0F0EBB1745
:10404000BC6BBBCAC0FA000195EC10F024300A0129
:10405000BC6F2330BB6FBC33BB33BC33BB33BC330F
:10406000BB330F0EBC17BB17BC6BBBCAC0FA000139
:1040700095EC10F023500F0B0A01BB6FBC6BC06FA7
:10408000000195EC10F026380A01BB6FBC6B0F0ED7
:10409000BB17BB17BC6BBBCAC0FA000195EC10F094
:1040A00026C0BBFA0A01BC6B0F0EBB17BC6BBBCAA8
:1040B000C0FA000195EC10F026300A01BC6F2530E3
:1040C000BB6FBC33BB33BC33BB33BC33BB330F0E12
:1040D000BC17BB17BC6BBBCAC0FA000195EC10F053
:1040E00025500F0B0A01BB6FBC6BC06F000195EC34
:1040F00010F0FF0E0A01C06F000195EC10F01CD00B
:104100000A01B7510F0B4009BB6FC06F000195EC5E
:1041100010F0080E0A01C06F000195EC10F0030EBC
:104120000A01C06F000195EC10F0FF0E0A01C06F8C
:10413000000195EC10F000D010D00A017E530DE084
:10414000020179517B5D06E17A517C5DD8A402D0F1
:104150000A0103D097988E980A01000158EF28F0C1
:10416000020179517B5D03E17A517C5D0CE07D0EAB
:104170007925E96E060E7A21EA6EEF3C04D085A817
:1041800002D097988E9800015CEF28F00A018E6BA0
:104190008451030804E185510308D8B484D08451C4
:1041A00003083EE08251885D03E184518A5D38E076
:1041B0008451000831E2845102082EE3825303E166
:1041C000010E826F05D08251180802E2180E826F2C
:1041D00082CA88FA84CA8AFA88CA8EFA8A51020880
:1041E00005E100016581659306D00A010001658340
:1041F00065910A018E6D02015F6B5E6B5D6B88CA13
:104200005CF25CC264F28ECAC7FA0A01C86B000194
:1042100074EC08F006D00A0188CA82FA8ACA84FAC5
:1042200000010A01855103083EE08351895D03E1E5
:1042300085518B5D38E08551000831E285510208D7
:104240002EE3835303E1010E836F05D083511408DD
:1042500002E2140E836F83CA89FA85CA8BFA89CA6F
:104260008EFA8B51020806E10001658765950A0107
:104270008E6D03D00001658565970201636B626BEB
:10428000616B89CA60F260C265F28ECAC7FA010E1C
:104290000A01C86F000174EC08F005D00A0189CA50
:1042A00083FA8BCA85FA000160EF28F00A01916B4E
:1042B000906B8F6B8E6B956B946B936B926B996B12
:1042C000986B976B966B9D6B9C6B9B6B9A6B28B8EE
:1042D00054D1226A216A206A1F6A2750000A00010D
:1042E00018E0010A5BE0030AD8B4A2D00A0AD8B4E5
:1042F0009FD00B0AD8B4CDD0070AD8B4D5D0010AC4
:10430000D8B4DED0030AD8B4FAD0010AD8B402D1A6
:1043100001D10A0E0A01C76FC86B0001C4EC09F095
:10432000080E0A01C76F010EC86F0001C4EC09F046
:10433000BC0E575C0A01966F7F0E5858976F000E9F
:104340005958986F000E5A58996F98CA9EFA97CA92
:104350009FFA96CAA0FA200ED16F98CAD2FA97CACD
:10436000D3FA96CAD4FA0001C7EC04F00A019D6B97
:104370009C6B9B6B010E9A6F9CCA9EFA9BCA9FFA1C
:104380009ACAA0FAD16B9CCAD2FA9BCAD3FA9ACA2B
:10439000D4FA0001C7EC04F02888EDD00A0E0A0117
:1043A000C76FC86B0001C4EC09F0080E0A01C76FA3
:1043B000010EC86F0001C4EC09F0BC0E57240A01BD
:1043C000966F7F0E5820976F000E5920986F000E41
:1043D0005A20996F98CA9EFA97CA9FFA96CAA0FA6D
:1043E000200ED16F98CAD2FA97CAD3FA96CAD4FAD5
:1043F0000001C7EC04F0010E5F5C0A019A6F000E29
:10440000000160590A019B6F9C6B9D6B9CCA9EFAD0
:104410009BCA9FFA9ACAA0FAD16B9CCAD2FA9BCACD
:10442000D3FA9ACAD4FA0001C7EC04F02888A3D0C2
:104430006FC2C7FA0A01C86B0001C4EC09F059C089
:104440009EFA58C09FFA57C0A0FA200E0A01D16FF9
:1044500059C0D2FA58C0D3FA57C0D4FA0001C7ECF9
:1044600004F070C2C7FA010E0A01C86F0001C4EC63
:1044700009F062C09EFA61C09FFA0A01D16BD26B4B
:1044800062C0D3FA61C0D4FA0001C7EC04F02888F6
:1044900072D00A0E0A01826F836F010E846F030EC1
:1044A000856F2888000167D00D0E0A01826F0A0E01
:1044B000836F020E846F030E856F288800015BD026
:1044C0000A0E0A01826F080E836F030E846F8A6FD3
:1044D000010E856F280ED16FD26BD36BD46B0001A8
:1044E000C7EC04F02A0E0A01D16FD26BD36BD46BE8
:1044F0000001C7EC04F06591659328883CD00A0E52
:104500000A01826F836F030E846F020E856F288805
:10451000000131D0280E0A01D16FD26BD36BD46B5E
:104520000001C7EC04F0080E0A01D16FD26BD36B07
:10453000D46B0001C7EC04F02A0E0A01D16FD26BD4
:10454000D36BD46B0001C7EC04F00A0E0A01D16FE3
:10455000D26BD36BD46B0001C7EC04F0030E0A01DD
:104560008A6F846F8B6F856F000165916593659588
:104570006597288800D070D10A012750000A0001F1
:1045800019E0010AD8B47FD0030AD8B4EAD00A0AE5
:10459000D8B4E7D00B0AD8B43FD1070AD8B43CD17D
:1045A000010AD8B439D1030AD8B436D1010AD8B433
:1045B00043D132D1230E0A01D16FD26BD36BD46BAE
:1045C0000001C7EC04F003C091FA02C090FA01C0E8
:1045D0008FFA00C08EFA0A0190AF02D0FF0E91133D
:1045E000030ED16FD26BD36BD46B0001C7EC04F018
:1045F00003C095FA02C094FA01C093FA00C092FA7F
:104600000A0194AF02D0FF0E9513BC0E575C966F53
:104610007F0E5858976F000E5958986F000E5A58D1
:10462000996F9D6B9C6B9B6B010E9A6F9151995D7D
:1046300029E30BE19051985D25E307E18F51975DE8
:1046400021E303E18E51965D1DE395519D5D1AE3D3
:104650000BE194519C5D16E307E193519B5D12E3DE
:1046600003E192519A5D0EE322520AE1215208E1E0
:104670002050060807E2FF0A03E11F50D00802E2BB
:10468000272A2898E9D0230E0A01D16FD26BD36B69
:10469000D46B0001C7EC04F003C091FA02C090FA99
:1046A00001C08FFA00C08EFA0A0190AF02D0FF0E4F
:1046B0009113030ED16FD26BD36BD46B0001C7EC97
:1046C00004F003C095FA02C094FA01C093FA00C046
:1046D00092FA0A0194AF02D0FF0E9513BC0E572434
:1046E000966F7F0E5820976F000E5920986F000E1E
:1046F0005A20996F010E5F5C9A6F000E000160599D
:104700000A019B6F9C6B9D6B9951915D29E30BE1B5
:104710009851905D25E307E197518F5D21E303E117
:1047200096518E5D1DE39D51955D1AE30BE19C5101
:10473000945D16E307E19B51935D12E303E19A5107
:10474000925D0EE322520AE1215208E12050060850
:1047500007E2FF0A03E11F50D00802E2272A289847
:104760007BD0230E0A01D16FD26BD36BD46B0001C7
:10477000C7EC04F003C091FA02C090FA01C08FFAAE
:1047800000C08EFA0A0190AF02D0FF0E9113030E03
:10479000D16FD26BD36BD46B0001C7EC04F003C0B4
:1047A00095FA02C094FA01C093FA00C092FA0A0185
:1047B00094AF02D0FF0E951357508E5D2CE15850E8
:1047C0008F5D29E15950905D26E15A50915D23E1BA
:1047D000000161510A01925D1EE1000162510A016E
:1047E000935D19E1945317E1955315E122520AE1C3
:1047F000215208E1205006080EE2FF0A03E11F5093
:10480000D00809E2272A2750080804E2232AD8B44E
:10481000242A276A289820D022520AE1215208E14E
:1048200020500E0807E2FF0A03E11F50A00802E231
:104830002898272A0A0110D022520AE1215208E1C1
:104840002050060807E2FF0A03E11F50D00802E2E9
:104850002898272A0A0100D0000167EF28F0F86A9B
:10486000D09E078E5E0E006E100E016E020EE96E77
:10487000000EEA6EEE6A002EFDD7012EFBD70A0E5F
:104880001E6EF10E1D6E040E0A01F26F6B0EF16FBB
:10489000F46BF36B0001EA6AE96A7C86A00E6F6E26
:1048A000010E7D6EA60E6C6E900E6B6E94869488D3
:1048B000500EC86E360EC66E226A216A206A1F6AC2
:1048C000246A236A266A256A276A286AFF0E496EC7
:1048D0004A904A82566A010E556E110E546E700E41
:1048E000536E5A6A596A880E586EB80E576E5E6AD1
:1048F0005D6A440E5C6E5C0E5B6E630E606F9C0EB8
:104900005F6E170E626F700E616F0B0E646FB80EE4
:10491000636F656B180E02015A6F140E5B6F5F6B4D
:104920005E6B5D6B5C6B636B626B616B606B646B2E
:10493000656B696B686B676B666B6D6B6C6B6B6BD8
:104940006A6B766B756B786B776B7A6B796B7C6B5C
:104950007B6B0A017D6B7E6B7F6B806BC150C00BE4
:104960000F09C16E070EB46E480E296E440E2A6EF2
:10497000320E2B6E300E2C6E5F0E2D6E4D0E2E6E87
:104980006F0E2F6E740E306E6F0E316E720E326EB1
:10499000336A560E346E300E356E310E366E2E0E74
:1049A000376E300E386E396E2E0E3A6E300E3B6E0C
:1049B000320E3C6E200E3D6E3E6A300E3F6E310E62
:1049C000406E2D0E416E410E426E700E436E720EA1
:1049D000446E2D0E456E310E466E476E486A100EBF
:1049E0000001666F050E676F040E686F030E696F36
:1049F000020E6A6F060E6B6F100E6C6F0D0E6D6FF0
:104A00000C0E6E6F0B0E6F6F0A0E706F2E0E716FA5
:104A1000100E726F050E736F040E746F030E756FB8
:104A2000020E766F060E776F100E786F0D0E796F8F
:104A30000C0E7A6F0B0E7B6F0A0E7C6F2E0E7D6F45
:104A4000100E7E6F050E7F6F040E806F030E816F58
:104A5000020E826F060E836F100E846F0D0E856F2F
:104A60000C0E866F0B0E876F0A0E886F2E0E896FE5
:104A7000110E8A6F8B6F8C6F8D6F8E6F8F6F906F33
:104A8000916F926F936F946F956F966F976F986F0A
:104A9000996F9A6F9B6F9C6F9D6F9E6F9F6FA06FBA
:104AA000A16FA26FA36FA46FA56FA66B010EA76F76
:104AB000020EA86F040EA96F050EAA6F060EAB6F4B
:104AC000080EAC6F090EAD6F0A0EAE6F0B0EAF6F16
:104AD0000D0EB06F0E0EB16F0F0EB26F100EB36FE2
:104AE000120EB46F130EB56F100EB66F110EB76FB6
:104AF000120EB86F130EB96F140EBA6F150EBB6F8E
:104B0000160EBC6F170EBD6F180EBE6F190EBF6F5D
:104B10001A0EC06F1B0EC16F1C0EC26F1D0EC36F2D
:104B20001E0EC46F1F0EC56F200EC66FC76F210EFD
:104B3000C86F220EC96F230ECA6F240ECB6F250ECD
:104B4000CC6F260ECD6F270ECE6F280ECF6F290E9D
:104B5000D06F2A0ED16F2B0ED26F2C0ED36F2D0E6D
:104B6000D46F2E0ED56F2F0ED66F300ED76F310E3D
:104B7000D86F320ED96F330EDA6F340EDB6F350E0D
:104B8000DC6F360EDD6F370EDE6F380EDF6F390EDD
:104B9000E06F3A0EE16F3B0EE26F3C0EE36F3D0EAD
:104BA000E46F3E0EE56FE66BE76BC80EE86FE96BEE
:104BB000E30EEA6FEB6BFF0EEC6FED6B1A0EEE6F10
:104BC000010EEF6F360EF06F010EF16F510EF26FA6
:104BD000010EF36F6D0EF46F010EF56F880EF66F18
:104BE000010EF76FA40EF86F010EF96FBF0EFA6F8A
:104BF000010EFB6FDB0EFC6F010EFD6FF70EFE6FFB
:104C0000010EFF6FC80E0101006F016B450E026FB0
:104C1000010E036FC20E046F010E056F3F0E066F8B
:104C2000020E076FBC0E086F020E096F390E0A6F75
:104C3000030E0B6FB60E0C6F030E0D6F330E0E6F5F
:104C4000040E0F6FB00E106F040E116F2D0E126F49
:104C5000050E136FAA0E146F050E156F270E166F33
:104C6000060E176F186B196BC80E1A6F1B6BE30ECD
:104C70001C6F1D6BFF0E1E6F1F6B1A0E206F010E37
:104C8000216F360E226F010E236F510E246F010E1D
:104C9000256F6D0E266F010E276F880E286F010E8F
:104CA000296FA40E2A6F010E2B6FBF0E2C6F010E01
:104CB0002D6FDB0E2E6F010E2F6FF70E306F010E72
:104CC000316F120E326F020E336F2D0E346F020EE3
:104CD000356F490E366F020E376F640E386F020E55
:104CE000396F800E3A6F020E3B6F9B0E3C6F020EC7
:104CF0003D6FB70E3E6F020E3F6FD20E406F020E39
:104D0000416FEE0E426F020E436F090E446F030EA9
:104D1000456F250E466F030E476F400E486F030E1A
:104D2000496F4A6B140E4B6F4C6F4D6F4E6F4F6F48
:104D30001E0E506F516F526F280E536F546F556F88
:104D4000320E566F576F586F596F5A6F5B6F5C6FAB
:104D50005D6F5E6F5F6F606F616F626F636B980E08
:104D6000646F656F666F676F686FE40E696F6A6F77
:104D7000800E6B6F6C6F6D6F6E6F6F6FBE0E706FAE
:104D8000716F726F736F746F756F766F776F786F07
:104D9000796F7A6F7B6F7C6B7D6B7E6B7F6B806BCB
:104DA000816B826B836B846B856B866B876B886B87
:104DB000010E896F8A6F8B6F8C6F8D6F8E6F8F6F07
:104DC000906F916F926F936F946F956B070E966FC4
:104DD000976F986F996F9A6F9B6F9C6F9D6F9E6F87
:104DE0009F6FA06FA16F050EA26FA36FA46FA56F39
:104DF000A66FA76FA86FA96FAA6FAB6FAC6FAD6FEF
:104E0000AE6BAF6BC80EB06FB16BE90EB26FB36B28
:104E1000090EB46F010EB56F2C0EB66F010EB76F91
:104E20004A0EB86F010EB96F6A0EBA6F010EBB6FF2
:104E30008B0EBC6F010EBD6FAB0EBE6F010EBF6F50
:104E4000CC0EC06F010EC16FEC0EC26F010EC36FAE
:104E5000C80EC46FC56B5E0EC66F010EC76FF40E31
:104E6000C86F010EC96F8A0ECA6F020ECB6F200E7B
:104E7000CC6F030ECD6FB60ECE6F030ECF6F4C0E00
:104E8000D06F040ED16FE20ED26F040ED36F780E86
:104E9000D46F050ED56F0E0ED66F060ED76FD86B7A
:104EA000D96BC80EDA6FDB6BE90EDC6FDD6B090EB8
:104EB000DE6F010EDF6F2C0EE06F010EE16F4A0E08
:104EC000E26F010EE36F6A0EE46F010EE56F8B0E69
:104ED000E66F010EE76FAB0EE86F010EE96FCC0EC7
:104EE000EA6F010EEB6FEC0EEC6F010EED6F0D0E25
:104EF000EE6F020EEF6F3F0EF06F020EF16F4E0E6F
:104F0000F26F020EF36F6E0EF46F020EF56F8F0EDE
:104F1000F66F020EF76FAF0EF86F020EF96FD00E3C
:104F2000FA6F020EFB6FF00EFC6F020EFD6F110E9A
:104F3000FE6F030EFF6F310E0201006F030E016F53
:104F4000026B140E036F046F056F066F1E0E076F62
:104F5000086F096F280E0A6F0B6F0C6F320E0D6F02
:104F60000E6F0F6F106F116F126F136F146F156F3D
:104F7000166F176B980E186F196F1A6F1B6FE40E70
:104F80001C6F1D6F1E6F800E1F6F206F216FBE0E76
:104F9000226F236F246F256F266F276F286F296F6D
:104FA0002A6F2B6F2C6B2D6B2E6B2F6B306B316B35
:104FB000326B336B346B356B366B010E376F386F7A
:104FC000396F3A6F3B6F3C6F3D6F3E6F3F6F406F85
:104FD000416B070E426F436F446F456F466F476FDB
:104FE000486F496F4A6F4B6F050E4C6F4D6F4E6F98
:104FF0004F6F506F516F526F536F546F556F566BA9
:10500000576B586B596B0A01816B826B836B030E74
:10501000846F856F866B876B886B896B8A6F8B6FEC
:105020008C6B8D6B97968E8697988E888C849594D2
:105030008C869596978A8D6B85BA8D2B978C8D6B08
:1050400085BC8D2B800ED56E00016CEF03F09D8624
:10505000C00EF212ECEC04F0640E0A01C86F0001FD
:10506000D2EC05F024EF06F0012C01D002D0C9EFFC
:1050700006F0DFEF07F0A2EC0AF097968E96246A0E
:10508000236A266A256A286A4A90FDEC0DF085BCE1
:105090000AD00A018D2B8D51640803E28D6B959423
:1050A0008C7403D000018C849594000139EF14F0C6
:1050B000FDEC0DF0B0EF20F0FDEC0DF0C6EF20F0B0
:1050C00085BA01D0FF0028520AE056EF21F0010E08
:1050D0001F26D8B0202AD8B4212AD8B4222AD5D75E
:0250E0000300CB
:020000040030CA
:0E00000000C2161E0305B100FFC0FFE0FF4066
:00000001FF
